:100000000C94D2050C9477240C940A060C940A06DE
:100010000C940A060C940A060C940A060C940A0620
:100020000C940A060C940A060C94A52C0C94772DBB
:100030000C94BF260C940A060C940A060C940A062B
:100040000C940A060C940A060C940A060C940A06F0
:100050000C940A060C9463270C940A060C940A0666
:100060000C940A060C940A060C940A060C940A06D0
:100070000C940A060C940A060C940A060C940A06C0
:100080000C940A060C940A060C940A060C940A06B0
:100090000C940A060C940A060C940A060C940A06A0
:1000A0000C940A060C940A060C940A06C509C509A4
:1000B000F109F109590A770A8F0B8F0B820A1B0B82
:1000C0002C0B2C0BE42D0B2E032F0B2E032F572E56
:1000D0007A2E032FD12EE02E290014001A000800DA
:1000E00015001700E00004001600070009000A00D0
:1000F000E1001D001B0006001900050003512B0044
:10010000E300E20002512C001C0018000C00120059
:1001100013002A000B000D000E000F003300340006
:100120001100100036003700380028002C00015163
:100130002B004C004600035101001E001F00200050
:10014000210022000100350038002F0026022D007A
:100150000100350238022F0200002D0201000100CB
:1001600001000100010001002300240025002600F9
:10017000270001002E00270230003100000001009E
:100180002E020000300231020100010001000100D6
:1001900001000100010001000100000000004B000F
:1001A00000000000010000004A004E004D00000069
:1001B00001000000500900004F090000010001008B
:1001C00001000100010001000000000052000000D9
:1001D000000001000000500051004F00000001002D
:1001E00000002B0300002B010000010001000100B2
:1001F0000100010001000100005C00003A003B002A
:100200003C000000010000003D003E003F000000F7
:1002100001000000AA000000A90000000100010088
:100220000100010001000100000040004100420007
:100230000000005C00004300440045000000010095
:100240000000AC00AE00AB000000010001000100A6
:10025000010001000100010044454255473A206475
:10026000697361626C65642E0A0044454255473AE1
:1002700020656E61626C65642E0A000A00253032CA
:1002800058006C65645F7461736B3A20004F6E6553
:1002900073686F743A206163746976653A202564E7
:1002A0000A000A0025303862003A20002530325812
:1002B000000A722F632030313233343536370A006A
:1002C00054617267657420636F6E6E6563746564F4
:1002D0000D0A0054617267657420646973636F6E00
:1002E0006E65637465642C207468726F74746C69D5
:1002F0006E6720636F6E6E656374696F6E206174E4
:1003000074656D7074730D0A004661696C656420D4
:10031000746F20657865637574652025730A0029FC
:100320000A002575002F002575005D280025640052
:100330002000256400200025640020002564007C46
:100340000025303258006D6F7573656B6579205BE1
:1003500062746E7C782079207620685D28726570E2
:100360002F61636C293A205B00313A0964656C6146
:1003700079282A31306D73293A2025750A323A09D5
:10038000696E74657276616C286D73293A202575E3
:100390000A333A096D61785F73706565643A2025A8
:1003A000750A343A0974696D655F746F5F6D6178C1
:1003B0003A2025750A353A09776865656C5F6D6185
:1003C000785F73706565643A2025750A363A097757
:1003D0006865656C5F74696D655F746F5F6D61788A
:1003E0003A2025750A00703A097072696E74207699
:1003F000616C7565730A643A097365742064656697
:1004000061756C74730A75703A092B310A646E3A1F
:10041000092D310A6C743A092B31300A72743A0989
:100420002D31300A4553432F713A09717569740AA9
:100430000A7370656564203D2064656C7461202AD0
:10044000206D61785F7370656564202A202872656D
:1004500070656174202F2074696D655F746F5F6DC6
:100460006178290A77686572652064656C74613A01
:1004700020637572736F723D25642C207768656503
:100480006C3D25640A53656520687474703A2F2F9B
:10049000656E2E77696B6970656469612E6F72672E
:1004A0002F77696B692F4D6F7573655F6B65797316
:1004B0000A004D3E20004D25753A25733E20003F31
:1004C0000A003D2025750A003F0A006465666175D3
:1004D0006C74730A0025750A003F0A000A092D2072
:1004E00056616C756573202D0A00710A000A092D8A
:1004F000204D6F7573656B6579202D0A003F0043B1
:100500003E20004C25640A000A092D2053746174B2
:100510007573202D0A686F73745F6B6579626F6104
:1005200072645F6C65647328293A20253032580A5A
:100530006B6579626F6172645F70726F746F636F05
:100540006C3A20253032580A6B6579626F617264AB
:100550005F69646C653A20253032580A74696D65AC
:10056000725F72656164333228293A202530386C15
:10057000580A000A092D2056657273696F6E202D86
:100580000A5649443A203078413130332861693085
:10059000332044657369676E2053747564696F29ED
:1005A000205049443A20307830303134284F72623C
:1005B00069745829205645523A203078303030310D
:1005C0000A4255494C443A20202846656220323779
:1005D0002032303232290A4F5054494F4E533A207C
:1005E0004C554641204D4F5553454B455920455894
:1005F0005452414B455920434F4E534F4C45204395
:100600004F4D4D414E4420343039360A4743433A2A
:1006100020352E342E30204156522D4C4942433A3B
:1006200020322E302E30204156525F415243483AFC
:1006300020617672350A000A092D20436F6E736FB0
:100640006C65202D0A4553432F713A097175697401
:100650000A6D3A096D6F7573656B65790A000A0951
:100660002D204D61676963202D0A443A0944656273
:100670007567204D65737361676520546F67676C9C
:10068000650A583A094D617472697820446562754B
:1006900067204D6F646520546F67676C65202D205F
:1006A00053686F77206B657970726573736573201B
:1006B000696E206D617472697820677269640A4B93
:1006C0003A094B6579626F617264204465627567AF
:1006D00020546F67676C65202D2053686F77206BFF
:1006E00065797072657373207265706F72740A4DEC
:1006F0003A094465627567204D6F75736520546FC4
:1007000067676C650A563A0956657273696F6E0AB7
:10071000533A095374617475730A433A0941637417
:10072000697661746520436F6E736F6C65204D6FE1
:1007300064650A46312D4631303A0953776974634E
:100740006820746F204C6179657220302D39202823
:10075000463130203D204C30290A302D393A09539A
:10076000776974636820746F204C617965722030FA
:100770002D390A47524156453A09537769746368DF
:1007800020746F204C6179657220302028616C7470
:1007900065726E617465290A423A094A756D702066
:1007A000746F20426F6F746C6F616465720A455399
:1007B000433A094A756D7020746F20426F6F746CF4
:1007C0006F616465722028616C7465726E61746516
:1007D000290A453A095072696E7420454550524FB6
:1007E0004D2053657474696E67730A4253504143D8
:1007F000453A09436C65617220454550524F4D0A98
:10080000006B65796D61705F636F6E6669672E72EC
:1008100061773A20253032580A2E737761705F6312
:100820006F6E74726F6C5F636170736C6F636B3A41
:100830002025750A2E636170736C6F636B5F746F34
:100840005F636F6E74726F6C3A2025750A2E737732
:1008500061705F6C63746C5F6C6775693A202575B5
:100860000A2E737761705F7263746C5F726775696B
:100870003A2025750A2E737761705F6C616C745F26
:100880006C6775693A2025750A2E737761705F72FF
:10089000616C745F726775693A2025750A2E6E6FF8
:1008A0005F6775693A2025750A2E737761705F67F7
:1008B000726176655F6573633A2025750A2E7377DA
:1008C00061705F6261636B736C6173685F626163C7
:1008D0006B73706163653A2025750A2E6E6B726FBB
:1008E0003A2025750A0064656275675F636F6E66FE
:1008F00069672E7261773A20253032580A2E656E6C
:1009000061626C653A2025750A2E6D617472697892
:100910003A2025750A2E6B6579626F6172643A2000
:1009200025750A2E6D6F7573653A2025750A006569
:1009300065636F6E6669673A0A64656661756C74B3
:100940005F6C617965723A2025750A003F000A6D77
:100950006F7573653A206F66660A000A6D6F75736E
:10096000653A206F6E0A000A6B6579626F61726486
:100970003A206F66660A000A6B6579626F6172647D
:100980003A206F6E0A000A6D61747269783A206FBE
:1009900066660A000A6D61747269783A206F6E0AA1
:1009A000000A64656275673A206F66660A000A6429
:1009B000656275673A206F6E0A000A0A4A756D70A3
:1009C000696E6720746F20626F6F746C6F6164650D
:1009D000722E2E2E2000433E2000436C656172690A
:1009E0006E6720454550524F4D0A000A00253032AF
:1009F0005820006B6579626F6172645F7265706F19
:100A000072743A20005B735D005B575D005B535D61
:100A1000005B525D005B445D005B435D000E034F75
:100A20000072006200690074005800000026036133
:100A30000069003000330020004400650073006945
:100A40000067006E002000530074007500640069A8
:100A5000006F0000000403090409025B00030100A9
:100A6000A0FA09040000010301010009211101009D
:100A7000012240000705810308000109040100016B
:100A800003000000092111010001227B00070582FB
:100A900003200001090402000203000000092111E3
:100AA000010001222200070583032000010705033E
:100AB00003200001120100020000000803A114003D
:100AC0000100010200010631FF0974A10109751539
:100AD0000026FF009520750881020976150026FF83
:100AE00000952075089102C005010902A101850247
:100AF0000901A1000509190129081500250195081A
:100B0000750181020501093009311581257F9502A2
:100B10007508810609381581257F950175088106BC
:100B2000050C0A38021581257F950175088106C0DC
:100B3000C005010980A101850319012AB70015012B
:100B400026B700950175108100C0050C0901A101AF
:100B5000850419012AA002150126A002950175102D
:100B60008100C005010906A101050719E029E71563
:100B7000002501950875018102950175088101051F
:100B800007190029FF150026FF009506750881004A
:100B9000050819012905950575019102950175034F
:100BA0009101C00011241FBECFEFDAE0DEBFCDBF40
:100BB00004B603FE18C080912F0390913003A091DA
:100BC0003103B09132038730904BA740B04B59F4BA
:100BD00010922F03109230031092310310923203BF
:100BE000E0E0F8E3099512E0A0E0B1E0EAEAFFE511
:100BF00002C005900D92AE32B107D9F723E0AEE204
:100C0000B2E001C01D92AF32B207E1F70E94361B7D
:100C10000C94D32F0C940000FF93EF93E0912E02DD
:100C2000F0912F02309709F00995EF91FF91089507
:100C3000FC018591803011F0EFDFFBCF0895FF2795
:100C4000E0E230E247FF0CC0419597FF09C0EDE2BA
:100C50006095709580959095611D711D811D911D08
:100C600027FF02C0219530E350E2AA27660F771FC5
:100C7000881F991FAA1FA41710F0A41B63955A95EB
:100C8000A9F7AA3008F0A95FA05DAF93F3956115AD
:100C900071058105910541F7ED3211F4EF93F3955C
:100CA000F21718F43F93F395FBCF8F91B5DFFA95C8
:100CB000E1F70895E991F9918591803021F085322D
:100CC00019F0AADFF9CF089520E0E8945591553244
:100CD000C1F3503311F4689455915A3348F450538A
:100CE00090F3220F022E220F220F200D250FF4CF9A
:100CF0000EF4219589919991533619F3533729F1BF
:100D0000533559F1BC0188279927E8945C3621F4C2
:100D10008991999168945591543639F446EF7EF053
:100D200077FF0DC08FEF9FEF0AC055374AE039F0CB
:100D3000583540E121F0523642E009F00895FF9322
:100D4000EF937DDFEF91FF91B7CFFF93EF93FC011E
:100D500081918030B9F360DFFBCFFF93EF9368DFC1
:100D6000F1CFDF93CF93CDB7DEB72596A3DFCF9139
:100D7000DF91089581E0089581E008950C94BC0608
:100D800008950C94C0061F93CF93DF9300D000D03A
:100D90001F92CDB7DEB749835A836B8330913102FE
:100DA00089819A81311114C0662359F0222349F0B8
:100DB0000E94CE0D182F682F89819A810E94750D8F
:100DC00003C00E94A10D182F69817A81812F04C070
:100DD0000E94CE0D69817A810F900F900F900F9035
:100DE0000F90DF91CF911F910C940B15FC01262FD2
:100DF000408151816281738184810C94C30681E0BA
:100E00000895CF93DF93EC0160E00E94F606BE01E7
:100E1000DF91CF910C94C1060C94D2160C94CE168F
:100E200008950E941F0C0E9410072FEF84E39CE09E
:100E3000215080409040E1F700C000000C948927C9
:100E40000F931F93CF93DF938C0161E00E94F6060E
:100E5000EC01B8010E94BE06882309F45BC0B8010A
:100E6000CE010E948423882309F454C0B801CE0126
:100E70000E94661E882309F44DC0B801CE010E946D
:100E8000E022882309F446C0F80182818823D9F141
:100E9000CF3D8CE5D80779F140F4C115FCE5DF07BB
:100EA00091F0C130DC4591F02EC0CC35EDE5DE0788
:100EB00041F1CD35FDE5DF0709F1CB35DD4519F50C
:100EC0000E94651220C00E94110724C08091B402C4
:100ED000C82FC095C170C0FB80F98093B402CC23A9
:100EE00029F08AE692E00E94180614C088E592E094
:100EF0000E94180610C00E9419130CC00E945C12B8
:100F000002C00E946812C801DF91CF911F910F911A
:100F10000C94BA06C0E08C2FDF91CF911F910F91F6
:100F200008950E94A2260C94BC070E94BF070C944F
:100F3000A8268295982F937344E0949F90011124E2
:100F40008C7C86958695282B822F8575880F2A7A2A
:100F50002695822B089508950C94AB0781E008959F
:100F60000C94AE070895CF93C82F0E94AC078C2F26
:100F70000E94B007CF91089580E00C94B3070E94BF
:100F8000A2250C94B307CF930E94A225C82F80916D
:100F90003002C81741F1C09330028091B40282FF41
:100FA0001EC080FF04C082E892E00E941806809173
:100FB000B40280FF0CC01F92CF938DE792E09F9305
:100FC0008F930E94B1060F900F900F900F90809119
:100FD000B40280FF04C08BE792E00E9418068C2FB9
:100FE000CF910C94B307CF910895CF93DF93CDB7F2
:100FF000DEB72B970FB6F894DEBF0FBECDBF4F8381
:10100000588769877A878B8761110E9494119E01A6
:101010002F5F3F4F86E0F90111928A95E9F785E04D
:10102000FE013796D90101900D928A95E1F78981E9
:101030009A814C815D81452B31F09F3F31F491E0E5
:101040008F3F19F403C091E001C090E090FF09C008
:1010500049815A816B817C818D819E810E94B5106E
:1010600005C0C9010E94FF068111F2CF2B960FB671
:10107000F894DEBF0FBECDBFDF91CF910895FC0184
:10108000808191810E94100E0895CF93882309F4E6
:10109000A9C0C82F8238C1F40E94A22581FDA2C038
:1010A00069E380910201909103010E947A260E94D7
:1010B000B6112FEF81EE94E0215080409040E1F78F
:1010C00000C0000069E319C0833801F50E94A22521
:1010D00080FD88C063E580910201909103010E9428
:1010E0007A260E94B6112FEF81EE94E021508040C5
:1010F0009040E1F700C0000063E58091020190910B
:1011000003010E947C26CF910C94B6118438C1F45F
:101110000E94A22582FD66C067E480910201909141
:1011200003010E947A260E94B6112FEF81EE94E00F
:10113000215080409040E1F700C0000067E4DDCF1F
:101140008CEF8C0F813AF8F48C2F0E948922811148
:1011500049C06C2F80910201909103010E944426A6
:10116000882349F06C2F80910201909103010E9425
:101170007C260E94B6116C2F809102019091030190
:101180000E947A26C0CF80E28C0F883048F4C77066
:1011900081E001C0880FCA95EAF70E947711B3CFAA
:1011A000EBE5EC0FE33040F4F0E0EC58FE4F8081CB
:1011B00090E0CF910C940C26E8E5EC0FE73150F469
:1011C000F0E0EE0FFF1FEA5BFE4F80819181CF912F
:1011D0000C942226CD3E30F08C2F0E94BB1BCF9169
:1011E0000C948D1CCF910895882309F464C0823833
:1011F00079F40E94A22581FF5EC069E3809102011B
:10120000909103010E947A260E94B61169E310C0F2
:101210008338B1F40E94A22580FF4DC063E5809120
:101220000201909103010E947A260E94B61163E5A3
:1012300080910201909103010E947C260C94B611CA
:10124000843879F40E94A22582FF35C067E480913A
:101250000201909103010E947A260E94B61167E470
:10126000E7CF9CEF980F913A10F4682FE1CF90E20E
:10127000980F983050F4877091E001C0990F8A95CB
:10128000EAF7892F0E947D11D9CF9BE5980F933003
:1012900020F480E090E00C940C2698E5980F9731AC
:1012A00020F480E090E00C9422268D3E20F00E94F5
:1012B000161C0C948D1C08951F93CF93DF93182F49
:1012C000EB010E944508209741F08FE99FE00197CC
:1012D000F1F700C000002197F6CF812FDF91CF9169
:1012E0001F910C94F408893319F060E070E002C09B
:1012F00060E570E00C945C09882321F00E9477116E
:101300000C94B6110895882321F00E947D110C944D
:10131000B6110895CF92DF92EF92FF920F931F9331
:10132000CF93DF937C01D62FC72FFC01128105815B
:1013300002950F700E946D118823B9F01123A9F056
:101340008C2F807F803421F080E28D0F883068F010
:1013500080910B0382FD09C082E00E9416120E9458
:101360006D1191E0D82ED92601C0D12CCC2EC2947B
:101370008FE0C8228C2D90E08C30910508F0CFC111
:10138000FC01EA5AFF4F0C94612F8C2F807FCF70A5
:10139000882311F0C295C07F112399F0CC2309F462
:1013A000AAC180E28D0F883010F0D11104C08C2FBB
:1013B0000E94771103C08C2F0E9487110E94B611E2
:1013C0009AC18D2F0E94F408CC2309F4A8C180E2B1
:1013D0008D0F883038F1DD2329F18C2F0E948D117B
:1013E00024C08C2F807FCF70803211F0C295C07FD7
:1013F000DD2319F0D130A1F13DC080910B0382FFB4
:1014000017C0112349F0CC2329F08C2F0E947711AB
:101410000E94B61180E070C180E00E94F408CC23E5
:1014200009F47DC18C2F0E947D110E94B61177C1F5
:10143000112371F0002341F0013031F40E94971123
:101440008C2B0E949F116BC10E9497118C2B1DC089
:10145000002319F0013009F462C10E94AC1125C0CB
:10146000112321F0063008F05AC10EC0053008F0F3
:1014700056C11BC0112361F0002331F0F7018581B3
:1014800080FF39C18F7085838C2F0E947C0947C1F2
:10149000002359F0D93309F03FC1FFEF07EE13E005
:1014A000F15000401040E1F735C18C2F0E948309B4
:1014B00036C18C2F86958695837019F0813061F046
:1014C0002EC1112321F08D2F9C2F937002C080E03C
:1014D00090E00E940C262BC1112321F08D2F9C2F10
:1014E000937002C080E090E00E94222620C18D2FE0
:1014F000112319F00E94BB1B02C00E94161C0E94FF
:101500008D1C15C18C2F837009F047C011110BC1C0
:101510002D2F229526952770220F220F6D2F6F7089
:10152000862F90E0A0E0B0E0022E04C0880F991F43
:10153000AA1FBB1F0A94D2F7D4FF10C04FE050E09F
:1015400060E070E004C0440F551F661F771F2A95A6
:10155000D2F7409550956095709503C040E050E0FB
:10156000BA01C695C695C3708A019B01082B192B39
:101570002A2B3B2BC901B801C23049F058F4C130C5
:1015800019F00E948B0CCFC00E94790CCCC00E9435
:101590009D0CC9C00E94770CC6C0112319F08C2F76
:1015A000817001C08695882309F4BDC02D2F229536
:1015B00026952770220F220F6D2F6F70862F90E0D7
:1015C000A0E0B0E0022E04C0880F991FAA1FBB1F25
:1015D0000A94D2F7D4FF10C04FE050E060E070E012
:1015E00004C0440F551F661F771F2A95D2F74095F8
:1015F00050956095709503C040E050E0BA01C695E3
:10160000C695C3708A019B01082B192B2A2B3B2BF3
:10161000C901B801C23049F058F4C13019F00E9434
:10162000500D81C00E943E0D7EC00E94620D7BC0A5
:101630000E94B10C78C0CF70112339F08C2F0E941A
:10164000D70C8D2F0E947C096EC08D2F0E948309BC
:101650008C2F0E94F80C67C0D23F21F128F4D03FB4
:1016600041F0D13FC1F043C0D33F19F1D43F79F0ED
:101670003EC0112341F0053008F051C08C2F8F710E
:101680000E941D0D4CC0063008F049C0F7CF809174
:101690000B0382FF18C0112339F08C2F8F710E9429
:1016A000D70C3DC01123C9F38C2F8F710E94F80C09
:1016B00036C0112329F08C2F8F710E94C20C2FC0CD
:1016C0000E94BD0C2CC0112349F0CF718C2F0E94B9
:1016D000D70C63E08C2F0E94FB1121C081E00E9497
:1016E00016120230E0F082E00E94161218C0112398
:1016F00031F0002391F28D2F0E94450810C0002385
:1017000099F2D93349F41FEF27EE33E0115020400E
:101710003040E1F700C000008D2F0E94F40888EFF0
:101720008C0D843020F40E94A2250E94B307DD2096
:10173000C9F00E94691180FD15C0F70112820E9454
:1017400063110E94D70CC7010E94D30B0E94631142
:10175000DF91CF911F910F91FF90EF90DF90CF908D
:101760000C94F80CDF91CF911F910F91FF90EF90A7
:10177000DF90CF9008950F931F93CF93DF93EC01E9
:10178000688179818A810E941B0E8C010E94740DF0
:101790000E94650CB801CE010E948A09DF91CF91A9
:1017A0001F910F910895CF93DF93EC019881898168
:1017B0002B813C81232B31F08F3F31F481E09F3F1F
:1017C00019F403C081E001C080E080FD1DC0CE019E
:1017D0000E942007811110C00E946D118823A1F082
:1017E0008A81882389F080910B0382FD0DC082E0FD
:1017F000DF91CF910C941612CE010E94BB0BCE014B
:10180000DF91CF910C940107DF91CF91089580E093
:1018100090E00E940C2680E090E00E9422260E9428
:1018200094110E94B6110E94401E0C948D1C809150
:101830000201909103010E947E260C94070C0E94E5
:1018400084110C94170C92959F70963079F010F4D7
:10185000925001C09A50923068F4803F69F018F4B9
:10186000883E40F409C0843F29F406C0883E20F039
:10187000813F11F080E0089581E00895FC018081AE
:1018800091810E94100E0E94230C0895CF93DF9344
:1018900000D000D01F92CDB7DEB70F900F900F9001
:1018A0000F900F90DF91CF910895CF93DF9300D0E9
:1018B00000D000D0CDB7DEB726960FB6F894DEBFC5
:1018C0000FBECDBFDF91CF910895089508950C9478
:1018D000660C0C94670C0E94690C60935402709320
:1018E000550280935602909357020C94070C0C9467
:1018F0006B0C0F931F93009154021091550220918D
:10190000560230915702602B712B822B932B1F9123
:101910000F910C946B0C0F931F9300915402109134
:101920005502209156023091570260237123822381
:1019300093231F910F910C946B0C0F931F930091A5
:10194000540210915502209156023091570260279F
:101950007127822793271F910F910C946B0C0C9485
:10196000660C0E94AF0C60935002709351028093FA
:101970005202909353020C94070C60E070E0CB018C
:101980000C94B10C0F931F9341E050E060E070E0C5
:101990008A019B0104C0000F111F221F331F8A956B
:1019A000D2F7C901B8011F910F910C94B10C0F939C
:1019B0001F9341E050E060E070E004C0440F551F09
:1019C000661F771F8A95D2F780915002909151023D
:1019D000A0915202B09153028A019B01082B192B4E
:1019E0002A2B3B2BC901B8011F910F910C94B10C0C
:1019F0000F931F9341E050E060E070E004C0440F9B
:101A0000551F661F771F8A95D2F7409550956095B0
:101A100070958091500290915102A0915202B09124
:101A200053028A019B01082319232A233B23C9015E
:101A3000B8011F910F910C94B10C0F931F9341E0CB
:101A400050E060E070E004C0440F551F661F771F30
:101A50008A95D2F78091500290915102A091520242
:101A6000B09153028A019B01082719272A273B2797
:101A7000C901B8011F910F910C94B10C0F931F93E2
:101A80000091500210915102209152023091530264
:101A9000602B712B822B932B1F910F910C94B10C07
:101AA0000F931F9300915002109151022091520206
:101AB0003091530260237123822393231F910F914E
:101AC0000C94B10C0F931F9300915002109151028E
:101AD0002091520230915302602771278227932769
:101AE0001F910F910C94B10C0895292F220F920F82
:101AF000990F890FE82FE695E695E695877051E0F6
:101B000001C0550F8A95EAF785E0E89FF00111249E
:101B1000EE5CFD4F20E030E070E04081CB01022E12
:101B200002C0969587950A94E2F781708195842783
:101B30008523842781932F5F3F4F2530310569F737
:101B40000895292F220F920F990F890F682F6695FC
:101B500066956695982F977085E0689FB00111246F
:101B600040E050E080E0FB01E40FF51FEE5CFD4F2C
:101B7000208130E0092E02C0369527950A94E2F7BD
:101B800021703327042E01C0220F0A94EAF7822B1A
:101B90004F5F5F4F4530510531F70895BF92CF92A7
:101BA000DF92EF92FF920F931F93CF93DF938C01FD
:101BB000C0905002D0905102E0905202F090530237
:101BC0008091540290915502A0915602B091570213
:101BD000C82AD92AEA2AFB2ACFE1D0E0D701C601D8
:101BE0000C2E04C0B695A795979587950A94D2F7C1
:101BF00080FD04C0219790F7B12C07C0BC2EB8011E
:101C00008C2F0E941E150197A9F38B2DDF91CF9188
:101C10001F910F91FF90EF90DF90CF90BF900895AC
:101C2000CF93DF93EC010E94CE0DBE010E941E15E2
:101C3000DF91CF9108951F93CF93DF93EB019091A4
:101C40003102992321F0CB010E94100E13C088238A
:101C500049F0CB010E94CE0D182F682FCE010E94B3
:101C6000750D04C0CB010E94A10D182FBE01812F5C
:101C70000E941E15DF91CF911F9108951F93CF935E
:101C8000DF93C091580216E080915902C81799F06D
:101C9000D0E01C9FF0011D9FF00D1124E65AFD4F6E
:101CA0004081518162817381848195810E94550CAC
:101CB0002196C770E9CFDF91CF911F910895409190
:101CC0008A0250918B0260918C0270918D028091FA
:101CD0008E0290918F020C94550CEF92FF920F930D
:101CE0001F93CF93DF9380918F0282958F7009F0BD
:101CF00065C080918C02882309F460C080915802ED
:101D0000F090590210918A0200918B0260918D022D
:101D100070918E0291E01F3F09F090E0C0910001A8
:101D2000D0910101292F96E0E92E8F1509F446C0C4
:101D30006115710521F00F3F21F030E003C031E063
:101D400001C0322F90E030FD36C0E89EF001E99EE0
:101D5000F00D1124DF01A65ABD4F11963C91119749
:101D6000301329C03C91311326C012963C91129732
:101D7000311121C013964D915C911497461B570B5E
:101D80004C175D07C0F480918F028F708061809343
:101D90008F02E15AFD4F80818F70806180838AE8D5
:101DA00092E00E94D30BDF91CF911F910F91FF9092
:101DB000EF900C943E0E01968770B7CFDF91CF91D4
:101DC0001F910F91FF90EF9008959F92AF92BF9255
:101DD000CF92DF92EF92FF920F931F93CF93DF93F7
:101DE000CDB7DEB761970FB6F894DEBF0FBECDBF9B
:101DF0008C0185E0F801DE011D9601900D928A9517
:101E0000E1F7D8011296EC9090918A02E0918B0252
:101E100020918D0230918E022115310531F0EF3F76
:101E200031F481E09F3F19F403C081E001C080E0FC
:101E3000B82FB1709B2E80FD47C1D8014C911196EF
:101E40005C9111971396AD90BC9014978AE8C82EB8
:101E500082E0D82EF0908C02B501621B730B2091AA
:101E6000000130910101FF2009F4D9C080918F0257
:101E70006217730708F095C0282F207F09F052C021
:101E80005E1313C0491311C0FE2CE1100EC08F70F9
:101E9000806180938F020E945F0EC6010E94D30B67
:101EA00080918F02F80185834DC1AB2831F05F3FEF
:101EB00031F481E04F3F19F403C081E001C080E0BC
:101EC00080FD03C081E08E2502C080E090E0F82F05
:101ED000F170FF2E80FF1CC08091580220915902A2
:101EE00036E0821709F40BC190E0389FF001399F6A
:101EF000F00D1124E65AFD4F6181561306C0608132
:101F0000461303C06281E61203C001968770E9CFD1
:101F1000FE2CEE2009F416C180918F02816080931F
:101F20008F0254C05E1306C0491304C0E11002C002
:101F3000F80199C0C8010E943E0C882361F1EE208F
:101F400051F120918F02822F82958F7090E002973D
:101F500074F080918A0290918B0298878F83198602
:101F6000BB86AA862C87CE0107960E94D30B86E0FB
:101F7000F801AAE8B2E001900D928A95E1F70E947B
:101F80006D0E0E945F0E0AC05E1711F1C8010E941B
:101F90003E0C81112CC0C8010E94D30BFF24F39486
:101FA000D1C0282F207F81F77A2DB98AA88A6E2D7B
:101FB00089890E94460C8AE892E00E94D30B86E051
:101FC000D6011D928A95E9F70E945F0EF12CBAC0E6
:101FD0004913DCCFE110DACFF8018583C8010E94F4
:101FE000D30B86E0D6011D928A95E9F7ABC0EE20AF
:101FF00091F220918F02822F82958F7090E002974C
:102000000CF4B5CF80918A0290918B029A838983D8
:102010001B82BD82AC822E83CE010196A6CF6217B1
:10202000730708F044C0FE2CEE2009F4B4CF5E1311
:1020300030C049132EC020918F0220FD21C0822F75
:1020400082958F70482F50E041155105C9F0F80175
:1020500025834F30510541F08F5F982F9295907FE7
:10206000822F8F70892B8583C8010E94D30B86E055
:10207000F801AAE8B2E001900D928A95E1F73CC020
:1020800086E0F801AAE8B2E001900D928A95E1F7A6
:1020900059C0C8010E943E0C811169CF80918F0206
:1020A000816080938F02C8010E94D30B4BC07A2DB0
:1020B000B98AA88A6E2D89890E94460C86E0D601CD
:1020C0001D928A95E9F718C0EE2009F464CFC80183
:1020D0000E943E0CF82E882309F45DCF86E0F801BB
:1020E000AAE8B2E001900D928A95E1F78AE892E0C1
:1020F0000E943F080E946D0E0E945F0E23C04D8714
:102100005E878D859E850E94100E292F22952F7047
:10211000223028F49F7039F0811105C00BC02430A3
:1021200028F49F7049F4805E883020F0C8010E9436
:10213000D30B9F2CF92C06C0D80115969C91907F4B
:1021400091F7F8CF8F2D61960FB6F894DEBF0FBED2
:10215000CDBFDF91CF911F910F91FF90EF90DF9056
:10216000CF90BF90AF909F9008951F93CF93DF9330
:10217000CDB7DEB72C970FB6F894DEBF0FBECDBF3C
:102180004F83588769877A878B879C87CE0107960C
:102190000E94E50E8823D1F09F8188852A853B85A2
:1021A000232B31F08F3F31F481E09F3F19F403C0BE
:1021B00081E001C080E080FD47C04F81588569857E
:1021C0007A858B859C850E94550C3EC086E0FE0179
:1021D0003796DE01119601900D928A95E1F7FF8105
:1021E000E8856A857B856115710531F0EF3F31F433
:1021F00081E0FF3F19F403C081E001C080E080FD71
:1022000023C02091590230E0C901019687709927B7
:102210004091580250E084179507F1F1F983EA8361
:102220007D836C8396E0929FD001939FB00D112423
:10223000A65ABD4FFE01319601900D929A95E1F795
:10224000809359020E943E0E16E0809158029091B0
:102250005902891771F1189FC0011124865A9D4FA8
:102260000E94E50E882329F1E09158021E9FF0019B
:102270001124E65AFD4F408151816281738184812E
:1022800095810E94550C8091580290E001968770CC
:10229000992780935802D9CF0E941F0C109259029F
:1022A00010925802EAE8F2E086E0DF011D928A957A
:1022B000E9F72C960FB6F894DEBF0FBECDBFDF91C5
:1022C000CF911F9108958091980285958595859568
:1022D0000895809198028770089590919802977060
:1022E00081E009F480E008958091A302089590911F
:1022F000A302892B8093A302089580959091A30255
:1023000089238093A30208951092A30208959091C7
:10231000A202892B8093A202089580959091A20237
:1023200089238093A20208951092A20208958091B9
:102330009902089508950C949A110C949B11909110
:102340000B0392FD08C090919902981721F0809399
:1023500099020C949D11089580919902882329F087
:102360001092990280E00C949D110895CF93DF9311
:10237000E0910201F09103018091A3028083E0913A
:102380000201F091030190818091A202892B808348
:1023900080919902882381F0E0910201F09103017C
:1023A0009081892B808380910201909103010E948A
:1023B000382681110E94AC11C0910201D091030115
:1023C00048E050E060E972E0CE010E947B2F892B4B
:1023D00069F088E0FE01A0E9B2E001900D928A95D3
:1023E000E1F7CE01DF91CF910C94B525DF91CF912C
:1023F00008950C949A1190910B0392FD10C098E0EF
:10240000899F90011124262B209398020E94D70CBB
:10241000809198028595859585950C94F9110C9479
:10242000D70C1092980280E00C94F9112091980238
:102430008095822380939802982F977099F430E0CA
:10244000482F082E000C550B2417350759F0909192
:102450000B0392FD07C08595859585950E94F80C24
:102460000C9411120895CF9390910B0392FB2227A5
:1024700020F92817F9F0C82F892FC0FB82F9809323
:102480000B0380910A0390910B030E94951282E046
:102490000E9416128091B40280FF0CC01F92CF934D
:1024A0008DE892E09F938F930E94B1060F900F905A
:1024B0000F900F90CF91089580910B0382FB882796
:1024C00080F991E089270C94331281E00C94331247
:1024D00080E00C9433126FEF7FEF80E090E00C947B
:1024E000BD2F80E090E00E94992F21E0893E9E4F11
:1024F00009F020E0822F089582E090E00C94912F63
:1025000083E090E00C94912FCF9384E090E00E94C0
:10251000912FC82F82E290E00E94912F2C2F30E063
:10252000A901582BCA01CF910895CF93C92F682FC5
:1025300084E090E00E949F2F6C2F82E290E0CF9188
:102540000C949F2FAB01BC018FE090E00C94B12F55
:10255000AB01BC0183E190E00C94B12F60E070E02E
:10256000CB010C94A81260E070E0CB010E94A21293
:102570000C94AE1269EE7EEF80E090E00E94BD2FD9
:1025800060E082E090E00E949F2F60E083E090E0B6
:102590000E949F2F109254021092550210925602E0
:1025A0001092570260E084E090E00E949F2F60E06C
:1025B00082E290E00E949F2F60E085E090E00E9420
:1025C0009F2F60E086E090E00E949F2F6FEF87E0F2
:1025D00090E00E949F2F40E050E0BA0188E090E038
:1025E0000E94B12F60E08DE090E00E949F2F40E0BC
:1025F00050E0BA0188E190E00E94B12F60E087E1ED
:1026000090E00E949F2F40E050E0BA018CE190E002
:102610000E94B12F60E070E080E290E00E94BD2F48
:1026200040E050E0BA0188E190E00E94B12F0C94A4
:10263000B3120C94BA12682F8EE090E00C949F2F86
:102640000E942C276093B0027093B1028093B20273
:102650009093B3026093AC027093AD028093AE028C
:102660009093AF02089585B7806885BF85B780686D
:1026700085BF08950C94BE1808950C943C130C94D7
:102680003C130C943F130C943C130C9443130C9484
:102690003C130E94331380E899E20E9498250E941F
:1026A00047130C9445130E943D130C943C130E9455
:1026B00053160C94B2070E9417270E94FA150E9425
:1026C000E1180E94D3170E9457130E944E1E0E94C9
:1026D000EB180C9441138F929F92AF92BF92CF92BE
:1026E000DF92EF92FF920F931F93CF93DF93CDB7BB
:1026F000DEB72A970FB6F894DEBF0FBECDBF0E949B
:102700002C18982E81110E94201384EAA82E82E0B2
:10271000B82E00E010E0802E802F0E947716D82E71
:10272000F501C1905F01C826B1F40F5F1F4F08305B
:10273000110589F78FEF89838A831B820E942027E6
:102740008160782F9D838C8349815A816B818D8133
:102750000E94F5072FC08091B40281FD0E947D1672
:10276000E12CFF24F3948C2D8F21F1F00E943A1379
:10277000882399F0EE828F82DF2081E009F480E0E7
:1027800088870E9420278160782F9A8789874E81C9
:102790005F8168858A850E94F507F801EC55FD4F39
:1027A0008081F826F08206C0E394FF0CF6E0EF1279
:1027B000DACFBBCF81E0911001C080E02A960FB63E
:1027C000F894DEBF0FBECDBFDF91CF911F910F9167
:1027D000FF90EF90DF90CF90BF90AF909F908F9041
:1027E00008950E946B130E94BE180E942D1D0C9428
:1027F000C307CF93DF930E942315EC01811521E5D8
:10280000920708F045C0811530E5930708F094C0A1
:10281000883E910528F5803E910508F0F8C0883A79
:10282000910570F4853A910508F07CC081309105DE
:1028300009F475C008F4E8C0049708F0E8C0E4C0E3
:102840008F3B910508F0E0C0C85AD0E0CC0FDD1FE7
:10285000C958DE4F0990D881C02DCE019464D8C0EC
:10286000811540E2940758F4811551E0950708F06E
:10287000CEC08D3E910508F4C7C09065C9C0C11592
:1028800080E4D80708F4C0C0DF70CE01906AC0C0F1
:10289000811525E59207A8F4811534E5930708F022
:1028A00095C0811543E5940708F07BC0811552E57A
:1028B000950708F061C0D82FCC27CE01816F906AB0
:1028C000A7C0C11589E5D807A0F4C11528E5D2072E
:1028D00008F082C0C11536E5D30708F095C08C2FEB
:1028E0000E94B7158F7190E0D82FCC27CE0190624F
:1028F0008FC0C1154AE5D40708F474C0CE019056C4
:102900008115904208F080C08D2F8F710E94B715FD
:10291000DD27D0628F71AE01582BCA0179C081E0EA
:1029200090E076C0C55AD0E0CB55DE4F8881C82FE5
:10293000D0E0CE0190646CC074E0969587957A954E
:10294000E1F7282F23703C2F337081E090E002C024
:10295000880F991F3A95E2F79C68AC01522B9A01B7
:102960009C2F9F709695969550E2959FE0011124BB
:10297000C9018C2B9D2B4CC08370992721E030E03E
:1029800002C0220F331F8A95E2F79C2F96959695E9
:1029900080E2989FE0011124C22BD32BCE019C68CA
:1029A00037C08370992721E030E002C0220F331F27
:1029B0008A95E2F79C2F9695969540E2949FE001C8
:1029C0001124C22BD32BCE019A6822C0D82FCC273A
:1029D000CE01846F906A1CC0DC2FCC27CE01806FA3
:1029E000906A16C08C2F8F700E94B71594E0D69510
:1029F000C7959A95E1F7CF70D0E0DC2FCC27D0694E
:102A00009E01282BC90104C080E090E001C0CE01E6
:102A1000DF91CF91089520E3829FC0011124FC0132
:102A200026E0729FE00DF11D1124E60FF11DEE0F5F
:102A3000FF1FE852FF4F8591949108950E940B1556
:102A40000E94F91308958238910569F1B0F4813339
:102A5000910509F46DC048F48932910509F463C009
:102A60008A32910509F469C008958533910509F406
:102A700055C089339105B9F00895833E910569F1F8
:102A800038F4803E9105B1F0823E910509F1089538
:102A9000863E9105A9F1873E9105B9F1843E9105E5
:102AA00009F064C023C020910A0320FD4FC021FD1E
:102AB0004DC0089580910A0380FD44C080910B03AE
:102AC00080FF44C080910A0384FD42C083EE4DC064
:102AD00080910A0382FF38C0F5CF80910A0382FDFE
:102AE00033C080910B0380FD31C0ECCF80910B038C
:102AF00081FF32C080910A0384FD2AC087EE35C071
:102B000080910A0383FF26C0F5CF80910A0383FDDD
:102B100021C080910B0381FD1FC0ECCF80910A037F
:102B200085FD1CC01DC080910A0385FD19C016C01B
:102B300080910A0386FD16C017C080910A0386FDA6
:102B400013C010C089E311C082EE0FC080EE0DC02B
:102B500080E00BC086EE09C084EE07C089E205C0A4
:102B600085E303C08AE201C081E390E0089590917B
:102B70000A0392FF0DC0282F2871283019F4877F8F
:102B8000846006C0282F2471243011F48B7F886064
:102B900093FF0DC0282F2871283119F4877E846196
:102BA00006C0282F2471243111F48B7E8861209176
:102BB0000B0320FF0DC0382F3871383019F4877F90
:102BC000816006C0382F3171313011F48E7F8860FA
:102BD00021FF0DC0282F2871283119F4877E8161CB
:102BE00006C0282F2171213111F48E7E886194FD59
:102BF000877E08951092060310920703109208032F
:102C0000109209030895CF92DF92EF92FF926B0129
:102C10007C010E94BE1881110EC00E942C27C61A8A
:102C2000D70AE80AF90AC0920603D0920703E09295
:102C30000803F0920903FF90EF90DF90CF90089582
:102C40000F931F930E94BE18882321F01F910F91AC
:102C50000C942C270E942C27009106031091070347
:102C60002091080330910903600F711F821F931F89
:102C70001F910F9108950C946B120E942C188FE3F2
:102C80009CE90197F1F700C000000E942C1880E039
:102C90000E94771680FF04C00E943B160C9489277F
:102CA00008950C943D160E947112811102C00E9479
:102CB00019130E947C128093B4020E948412909394
:102CC0000B0380930A030E9451160E948012682F02
:102CD00070E080E090E00E94770C6091500270916B
:102CE000510280915202909153020C94AF0CE82F44
:102CF000F0E0EB5EFC4F80810895CF92DF92EF927F
:102D0000FF920F931F93CF93DF9381EB92E00E948A
:102D1000180685E1E82E83E0F82EC0E0D0E09CEABA
:102D2000C92E92E0D92E04EA12E0DF93CF93DF920E
:102D3000CF920E94B10689EA92E00E941806F7013C
:102D400081917F010E9499071F928F931F930F9388
:102D50000E94B10682EA92E00E94180621968DB781
:102D60009EB708960FB6F8949EBF0FBE8DBFC830B1
:102D7000D105D9F6DF91CF911F910F91FF90EF9080
:102D8000DF90CF90089580EA8A95F1F7089500C00A
:102D900008950C94C31608950C94CB160C94CC167D
:102DA0000C94CB160C94D0160C94CB160F931F9347
:102DB000CF93DF9300D000D0CDB7DEB70E94BE180E
:102DC00060911D038823E9F119821A821B821C82FB
:102DD000862F90E08E010F5F1F4FB8018B5E9C4FD6
:102DE0000E94F918882389F080910C0390E044E058
:102DF00050E0B8018B5E9C4F0E947B2F21E0209316
:102E0000B502892B69F410E019C08091B5028823BE
:102E1000D1F384E0F80111928A95E9F71092B50296
:102E2000E0910C03F0E0EB5EFC4F89819A81AB816D
:102E3000BC8180839183A283B38311E00E940E073B
:102E40000DC070E06B5E7C4F80910C0390E08B5E58
:102E50009C4F0E9495190E94D41610E0812F0F906C
:102E60000F900F900F90DF91CF911F910F910895C8
:102E7000F894E82FE295EF70F0E031A1282F2F7041
:102E800081E090E001C0880F2A95EAF7982F90958D
:102E9000932391A392A1892B82A3789408950F93F1
:102EA0001F93CF93DF93CAE0D1E089918F3F11F058
:102EB0000E94381781E0CE30D807B9F7C4E0D1E0DE
:102EC0000AE011E089918F3F11F00E9438170C172A
:102ED0001D07C1F7DF91CF911F910F910895CF92F8
:102EE000DF92EF92FF920F931F93CF93DF938C01AA
:102EF000C62FD0E0CE01865F9E4F7C01FC01908101
:102F00009F3F09F447C0D62EF894E92FE295EF7061
:102F1000F0E081A19F7021E030E001C0220F9A957E
:102F2000EAF7822B81A382A12095282322A37894FB
:102F30000E94C716E4E0F1E04AE051E031E0C12C24
:102F400021912F3F89F0A22FA295AF70B0E090960B
:102F50008C9190E02F7002C0959587952A95E2F7A5
:102F600080FD02C0832F01C080E0C82A330F4E17B6
:102F70005F0731F7F70180818F3F11F00E9438170A
:102F800061E0C11001C060E08D2D0E94C916C00F24
:102F9000D11FC882DF91CF911F910F91FF90EF90C9
:102FA000DF90CF900895CF93DF9300D000D000D072
:102FB000CDB7DEB780910E01811124C030913C0164
:102FC00020913D0190913E0180913F0130930A0193
:102FD00020930B0190930C0180930D0186E0E0E4B7
:102FE000F1E0DE01119601900D928A95E1F7FE0164
:102FF0003196A4E0B1E0CE01079621912D938E1772
:103000009F07D9F780910E01811102C094E001C0A1
:1030100090E090931D0384E0891B80930C030E9431
:103020004F1788E0E5E1F3E0DF01982F1D929A95B4
:10303000E9F7EDE0F3E0DF011D928A95E9F784E01E
:103040000E94801826960FB6F894DEBF0FBECDBF43
:10305000DF91CF910C940C07EF92FF920F931F9387
:10306000CF93DF93CDB7DEB728970FB6F894DEBFC6
:103070000FBECDBF8E010F5F1F4F88E0F801119288
:103080008A95E9F7F12C6F2DC8010E946F17F39410
:10309000F4E0FF12F8CF48E050E0B8018DE093E093
:1030A0000E947B2F7C0121E0892B09F420E0E114B0
:1030B000F10441F088E0F801ADE0B3E001900D9239
:1030C0008A95E1F760911D0370E06B5E7C4F44E0F0
:1030D0008DE093E00E948118EF2819F40E94D61623
:1030E00002C081E090E028960FB6F894DEBF0FBED4
:1030F000CDBFDF91CF911F910F91FF90EF90089579
:103100000895FF920F931F93CF93DF938C01F62EB8
:10311000D72FC42F222349F081E08093B8020E9468
:1031200020279093B7028093B6028091B80288233B
:10313000C1F08091B6029091B7020E94382705979E
:1031400080F0EF2DFD2FD8014C2F50E0CD01801BDA
:10315000910B841795071CF48D918193F7CF1092F2
:10316000B802DF91CF911F910F91FF90089555986C
:103170005D9889B185FB882780F90895CF93809168
:10318000BB02811116C0CAEF0E943B2F81110AC0F9
:103190008FE39CE90197F1F700C00000C150A1F74F
:1031A00082E001C081E08093BB02823011F40E9472
:1031B000362F81E09091BB02913009F080E0CF91F1
:1031C00008950E94B71880930E010E94BE188111C5
:1031D0000C94431908950E94BE18811102C00C94EA
:1031E0004519089581E09091BC029A3008F080E082
:1031F0000895EF92FF920F931F93CF938C017B0161
:10320000C091BC02CA3038F4B701C8010E949319BA
:10321000811126C00AC08091B9029091BA020E9421
:103220003827843F914080F719C08091BC028F3FBE
:1032300019F08F5F8093BC028091BC028A30E0F06D
:103240000E9420279093BA028093B9028091B40221
:1032500080FF04C083ED92E00E94180680E00DC05C
:10326000CA3040F08091B40280FF04C080EC92E04C
:103270000E9418061092BC0281E0CF911F910F911D
:10328000FF90EF9008950C9431240C943424DF9235
:10329000EF92FF920F931F93CF93DF937901C82F83
:1032A000880FDD0B41155105A9F0FE0193E0EE0FEB
:1032B000FF1F9A95E1F7E15FFE4F81819281835470
:1032C0009D4F208130E04217530708F49A01A9016D
:1032D0000E94882FCE010E941D25D82E8823D1F070
:1032E00001151105B9F083E0CC0FDD1F8A95E1F7D8
:1032F000FE01E15FFE4F438150E00417150708F41B
:10330000A801C15FDE4F6C817D8163547D4FC70191
:103310000E94882F8D2DDF91CF911F910F91FF90EB
:10332000EF90DF9008950C94D01A0C94F01A0F933C
:103330001F93CF93DF9300D000D0CDB7DEB760915D
:10334000D2027091D3028091D4029091D5020E9452
:103350004727643671058105910528F10E942016E2
:10336000DC01CB010296A11DB11D89839A83AB8339
:10337000BC8300E010E020E030E044E050E0BE011B
:103380006F5F7F4F82E00E944719182F882361F0FA
:103390000E942C276093D2027093D3028093D402B0
:1033A0009093D50201C011E0812F0F900F900F90E4
:1033B0000F90DF91CF911F910F9108958F929F925F
:1033C000AF92BF92CF92DF92EF92FF920F931F9333
:1033D000CF93DF937C015B01942E852E69010E94BF
:1033E000F218811103C001E010E002C00AE010E011
:1033F000C1E0D0E0F894B501C701F60109957894D1
:10340000811129C021960C171D078CF0CC9F9001CB
:10341000CD9F300D300D112480E090E045E34A95BA
:10342000F1F70000019628173907C1F7E3CF909113
:10343000B402892F817090FF0FC08F929F9289E014
:1034400093E09F938F930E94B1060F900F900F907F
:103450000F9080E001C081E0DF91CF911F910F912B
:10346000FF90EF90DF90CF90BF90AF909F908F90A4
:103470000895AF92BF92CF92DF92EF92FF920F9397
:103480001F93CF93DF9300D000D01F92CDB7DEB74C
:103490005B01E090A801F090A90101E010E09E011D
:1034A0002B5F3F4F40E050E060E070E080E00E9422
:1034B0004719182F882309F43EC067018FEFC81AF7
:1034C000D80A6091CE027091CF028091D002909183
:1034D000D1020E944727643671058105910518F1D4
:1034E00004E010E09E012F5F3F4F40E050E060E0BD
:1034F00070E081E00E944719182F64E070E0C60177
:103500000E944F1E91E02D81281390E0192351F164
:103510000E942C276093CE027093CF028093D0023A
:103520009093D10211C064E070E0C6010E944F1E6A
:103530009D818913D5CFF70181819281A381B481C7
:1035400089839A83AB83BC83112361F089819A813B
:10355000AB81BC818093CA029093CB02A093CC0232
:10356000B093CD028091CA029091CB02A091CC027F
:10357000B091CD02F50180839183A283B383812F23
:103580000F900F900F900F900F90DF91CF911F91A0
:103590000F91FF90EF90DF90CF90BF90AF90089584
:1035A0000F931F93CF93DF93EC018B0129E33AE153
:1035B0004AEA51E00E94DE19882361F027E939E1E7
:1035C00047EB51E0B801CE01DF91CF911F910F91F0
:1035D0000C94DE1980E0DF91CF911F910F91089537
:1035E0000F931F93CF93DF93F894C091A801D091CC
:1035F000A901CE01019624E0FB01DC0101900D92AE
:103600002A95E1F764E070E00E944F1E8883789469
:10361000F8946D817E818F8198850091C60210910A
:10362000C7022091C8023091C90260177107820752
:10363000930751F06093C6027093C7028093C8024B
:103640009093C9020E9403167894DF91CF911F9145
:103650000F9108950E94FC290E945B130C94082A84
:103660000E940C2A0E94F1130C942A2A0E94BE2662
:103670000E94E3290E9449130E942A1B0E94301BCA
:103680000E945313FBCF8091DC0280FF06C0609143
:103690002C0170E0660F771F26C081FF04C0609187
:1036A0002C0184E005C082FF07C060912C0188E0F6
:1036B000689FB001112417C09091DB029923D1F0CB
:1036C00060912B01961788F720912C0188E0289FA4
:1036D00090011124929FA001939F500D112470E03E
:1036E000CA010E944D2F6038710540F461157105C3
:1036F00019F406C068E070E0862F08958FE70895FA
:1037000081E008958091DC0280FF08C0609128016B
:1037100070E0759567957595679521C081FF06C026
:103720006091280170E07595679519C082FF04C00B
:103730006091280170E010C09091DA02992399F00D
:10374000609127019617A0F780912801899FC001F9
:10375000112470E00E944D2F6038710540F461150E
:10376000710519F406C061E070E0862F08958FE7B7
:10377000089581E008958D3E21F40E94431B8195B8
:1037800004C08E3E29F40E94431B8093E0020895FA
:103790008F3E21F40E94431B819504C0803F29F491
:1037A0000E94431B8093DF020895893F19F40E9411
:1037B000821B05C08A3F31F40E94821B8195809351
:1037C000E10208958B3F21F40E94821B819504C081
:1037D0008C3F29F40E94821B8093E20208959FE0AF
:1037E000980F983078F421E030E0A90102C0440F2E
:1037F000551F9A95E2F7CA019091DE02892B8093BA
:10380000DE0208958D3F21F48091DC0281600BC0BF
:103810008E3F21F48091DC02826005C08F3F29F445
:103820008091DC0284608093DC0208958D3E39F43F
:103830009091E00297FF35C01092E00259C08E3E91
:1038400029F49091E0021916BCF32BC09091DF028D
:103850008F3E29F497FF25C01092DF0249C0803FB8
:1038600019F41916CCF31DC09091E102893F29F497
:103870001916BCF41092E1023BC08A3F19F497FF7D
:1038800010C0F8CF8B3F39F49091E20297FF09C046
:103890001092E2022DC08C3F21F49091E2021916A1
:1038A000BCF39FE0980F983080F421E030E0A9014C
:1038B00002C0440F551F9A95E2F7CA018095909176
:1038C000DE0289238093DE0213C08D3F21F48091B4
:1038D000DC028E7F0BC08E3F21F48091DC028D7F55
:1038E00005C08F3F29F48091DC028B7F8093DC023E
:1038F0008091DF02811106C08091E002811102C037
:103900001092DB028091E102811106C08091E202F7
:10391000811102C01092DA0208958091B40283FFEF
:103920007EC086E493E00E9418068091DE021F921A
:103930008F9381E493E09F938F930E94B1068FE36E
:1039400093E00E9418068091DF02282F082E000CB9
:10395000330B3F938F938CE393E09F938F930E945D
:10396000B1068AE393E00E9418068091E002282FB6
:10397000082E000C330B3F938F9387E393E09F93C4
:103980008F930E94B10685E393E00E941806809110
:10399000E102282F082E000C330B3F938F9382E314
:1039A00093E09F938F930E94B10680E393E00E947F
:1039B00018068091E202282F082E000C330B3F934B
:1039C0008F938DE293E09F938F930E94B1068AE2DA
:1039D00093E00E9418068091DB021F928F9387E28A
:1039E00093E09F938F930E94B10685E293E00E943B
:1039F00018068091DC021F928F9382E293E09F93DE
:103A00008F930E94B1068FE193E00E9418068DB754
:103A10009EB74C960FB6F8949EBF0FBE8DBF0E9406
:103A200020272091DF02211104C02091E0022223EF
:103A300021F09093D9028093D8022091E1022111C4
:103A400004C02091E202222321F09093D7028093B8
:103A5000D6028DED92E00C94FE25EF92FF920F932B
:103A60001F93CF93DF9300D000D000D0CDB7DEB747
:103A700086E0EDEDF2E0DE01119601900D928A955F
:103A8000E1F7E090DF02F090E0020091E102109196
:103A9000E2021092DF021092E0021092E102109214
:103AA000E202E11003C0FF2009F45DC08091D8025A
:103AB0009091D9020E943827AC019091DB029923A2
:103AC00039F020912D0130E02417350758F04BC014
:103AD00020912E018AE0289F900111242417350798
:103AE00018F041C09F3F19F09F5F9093DB02EE20DA
:103AF00061F00E94431B1E1414F09FEF01C091E07F
:103B0000989F902D11249093DF02FF2061F00E9476
:103B1000431B1F1414F09FEF01C091E0989F902D5C
:103B200011249093E0023091DF023323E1F02091E1
:103B3000E0022223C1F045EB3403C0011124992394
:103B400019F09093DF0203C081E08093DF0235EB30
:103B50002303C0011124992319F09093E00203C0BC
:103B600081E08093E002011103C0112309F45DC0DC
:103B70008091D6029091D7020E943827AC01909193
:103B8000DA02992339F02091290130E02417350712
:103B900058F04BC020912A018AE0289F90011124FF
:103BA0002417350718F041C09F3F19F09F5F90938D
:103BB000DA02002361F00E94821B101614F09FEFBE
:103BC00001C091E0989F902D11249093E102112360
:103BD00061F00E94821B111614F09FEF01C091E06A
:103BE000989F902D11249093E2023091E1023323AB
:103BF000E1F02091E2022223C1F045EB3403C00141
:103C00001124992319F09093E10203C081E080937D
:103C1000E10235EB2303C0011124992319F090939D
:103C2000E20203C081E08093E2028091DF02811111
:103C30000BC08091E002811107C08091E1028111E7
:103C400003C08091E20281110E948D1CEB82FC82F4
:103C50000D831E8386E0FE013196ADEDB2E001904A
:103C60000D928A95E1F726960FB6F894DEBF0FBE47
:103C7000CDBFDF91CF911F910F91FF90EF900895ED
:103C8000EDEDF2E086E0DF011D928A95E9F71092F2
:103C9000DB021092DA021092DC0208950895FC0112
:103CA000680F791F8FEF91E3E617F70771F0219105
:103CB000822728E030E087FF03C0880F892701C0F2
:103CC000880F21503109B9F7EFCF0895CF93DF93D3
:103CD000EC01FB018281882309F43CC1C430FDE57D
:103CE000DF0760F4CB3F9CE5D90788F49E012250A2
:103CF0003C452431310508F02EC109C0C236EDE53E
:103D0000DE0729F0C63AFDE5DF0709F024C10E946D
:103D1000841290930B0380930A03C1318CE5D8077A
:103D200009F4C6C008F042C0C930ECE5DE0709F46A
:103D30009BC000F5C5308CE5D80709F485C078F440
:103D4000C330ECE5DE0709F478C008F07AC0C23071
:103D5000DC4509F0F5C080910A038160EFC0C730EF
:103D60009CE5D90709F478C008F07AC080910A036D
:103D70008061E4C0CD30FCE5DF0709F487C058F46A
:103D8000CB309CE5D90709F479C008F07BC080915D
:103D90000A0388606FC0CF30FCE5DF0709F480C0FC
:103DA00008F082C080910A03877FC8C0CE3F9CE59F
:103DB000D90709F471C000F5C531FCE5DF0709F446
:103DC00085C068F4C3319CE5D90709F475C008F0D3
:103DD00095C00E941F0C80910A038F77AFC0CC3F23
:103DE000FCE5DF07A9F108F054C0CB3FDC4509F042
:103DF000A7C080910B0340C0C230EDE5DE0709F497
:103E000089C058F4C1158DE5D80709F45AC008F0E7
:103E100069C080910B0382602FC0C236EDE5DE07DA
:103E200009F47CC0C63AFDE5DF0709F481C0C33060
:103E3000DD4509F085C080E06EC080910A03826094
:103E40007DC080910A0316C080910A03886076C005
:103E500080910B0382604FC080910A0380626EC024
:103E600080910A0380646AC00E941F0C80910A033B
:103E7000806864C0846062C081603DC080910A0334
:103E80008E7F5CC080910A038D7F58C080910A03A9
:103E900016C080910B0318C080910B038D7F2BC03F
:103EA00080910A038F7E4AC080910A038F7D46C0AD
:103EB00080910A038F7B42C080910A03877F8B7FAA
:103EC0003DC080910B038D7F8E7F15C080910A03CA
:103ED00082FB222720F991E0922790FB82F990FB48
:103EE00083F92CC080910B03982F909591708E7F51
:103EF000892B90FB81F980930B0322C00E941F0C39
:103F000080910A0387FB222720F991E0922790FBFA
:103F100087F914C081E00E941B1312C080910A032C
:103F200084FB222720F991E0922790FB84F906C0B8
:103F300080910A03982F909590FB80F980930A0353
:103F400080910A0390910B030E9495120E941F0C0E
:103F500080E001C081E0DF91CF9108958091270139
:103F60001F928F93809128011F928F9380912B0134
:103F70001F928F9380912C011F928F9380912D011E
:103F80001F928F9380912E011F928F9389E693E069
:103F90009F938F930E94B1068DB79EB70E960FB672
:103FA000F8949EBF0FBE8DBF0895883220F58E31E4
:103FB00008F068C08B3091F1C0F4873009F0BEC0C2
:103FC00081E080932E0184E180932D018AE080932B
:103FD0002C018EE180932B0188E08093280188E2F8
:103FE000809327018BEC94E0C6C0833109F443C071
:103FF000843169F1A3C08F3409F49EC028F489325A
:1040000031F1883359F09AC0813531F008F4D4C0C9
:10401000823509F4A7C092C08FEFA5C08DEE94E061
:104020000E9418060E94AE1F1F9281E08F931F927C
:1040300088E08F9386EE93E09F938F930E94B10662
:104040000F900F900F900F900F900F9096C08AEEE8
:1040500094E00E9418068091E702882309F4AAC020
:104060001092E7021092E6021092E5021092E4022A
:104070001092E302B1C08CED94E00E9418060E94F9
:10408000AE1F7BC08D518093E702833031F170F415
:104090008130D1F0823009F03FC08DE291E0909301
:1040A000E6028093E5028FEC91E01FC0853059F164
:1040B00008F1863089F587E291E09093E6028093DB
:1040C000E5028AE092E011C08EE291E09093E60270
:1040D0008093E50286EC91E008C08CE291E0909339
:1040E000E6028093E5028BED91E09093E4028093E9
:1040F000E30218C08BE291E09093E6028093E50220
:1041000088EE91E0F2CF88E291E09093E60280930E
:10411000E50287EF91E0E9CF1092E70289ED94E0A4
:104120000E9418068091E702882309F455C01F9267
:104130008F9385ED94E00DC08AE015C088EC94E083
:104140001AC097FF47C0108280811F928F9382EC24
:1041500094E09F938F930E94B1060F900F900F9061
:104160000F900BC081E0E091E502F091E6023097FC
:1041700029F58FEB94E00E9418062091E702222394
:1041800059F18091E3029091E402009711F482ECDE
:1041900091E09F938F931F922F9386EB94E09F93D0
:1041A0008F930E94B1060F900F900F900F900F9079
:1041B0000F9016C080E0089586EFD5CF2081082E9D
:1041C000000C990B820F911D8F3F910509F00CF4A3
:1041D000B8CF8FEF8083B8CF82EB94E00E941806AF
:1041E00081E00895CF93C82F1F928F9383E095E0CD
:1041F0009F938F930E94B10681E090E0A0E0B0E031
:10420000BC01CD0104C0660F771F881F991FCA9596
:10421000D2F70E94770C0F900F900F900F90CF91D4
:104220000C941F0CEF92FF920F931F93CF93DF9389
:104230008B3109F4EDC008F08EC08B3009F4B1C0A9
:1042400008F078C0863009F4AFC020F4853009F456
:10425000BDC04EC1873009F4C0C0883009F048C1E4
:104260000E9480121F928F938FE299E09F938F9309
:104270000E94B1060E947C1283FB992790F91F923D
:104280009F9382FB992790F91F929F9381FB992717
:1042900090F91F929F93982F91701F929F931F9256
:1042A0008F9386EE98E09F938F930E94B1060E94B1
:1042B000841287FB222720F91F922F9386FB222747
:1042C00020F91F922F9385FB222720F91F922F930D
:1042D00084FB222720F91F922F9383FB222720F9AA
:1042E0001F922F9382FB222720F91F922F9391FB7D
:1042F000222720F91F922F93292F21701F922F938D
:1043000081FB222720F91F922F93282F21701F92C3
:104310002F939F938F9381E098E09F938F930E94B8
:10432000B1068DB79EB788960FB6F8949EBF0FBEA4
:104330008DBF35C0803109F495C020F48E3009F46A
:104340007BC0D6C0863109F4A8C0893109F0D0C03D
:1043500083E795E084C08A32E1F060F4873209F4A3
:10436000C3C028F48E3108F4C3C08D51BEC0893259
:1043700069F1BEC0833448F48A3308F0B3C0853392
:1043800009F4B2C0883369F0B3C0833409F4ACC017
:10439000AFC08AED99E00E9418060E941913C1E08F
:1043A000ACC08EE596E05BC08091B402817F8E7FC9
:1043B0008093B40287E396E00E94180686ED99E0A8
:1043C0000E94180681E08093E802E9CF8AEB99E029
:1043D0000E9418060E941107E2CF8091B402C82FF4
:1043E000C095C170C0FB80F98093B402CC2329F042
:1043F0008EEA99E00E94180680C081EA99E00E9446
:1044000018068091B402897F877F8093B402C7CF5A
:104410009091B40291FBCC27C0F981E0C827892F85
:10442000C0FB81F98093B402CC2319F084E999E0B0
:1044300029C086E899E013C09091B40292FBCC2782
:10444000C0F981E0C827892FC0FB82F98093B402AC
:10445000CC2319F087E799E015C087E699E00E9420
:1044600018069DCF9091B40293FBCC27C0F981E050
:10447000C827892FC0FB83F98093B402CC2351F065
:104480008BE599E00E9418068091B40281608093C8
:10449000B40233C08EE499E0E2CF0E942C27162F9D
:1044A000072FF82EE92ED0910503C0913B010E9401
:1044B000A225EF92FF920F931F931F92DF931F92FB
:1044C000CF931F928F9388E095E09F938F930E94E4
:1044D000B1068DB79EB70C960FB6F8949EBF0FBE6F
:1044E0008DBF5DCF895301C080E00E94F22057CF7D
:1044F0008CE499E00E941806C0E08C2FDF91CF91E8
:104500001F910F91FF90EF90089580E008950C9413
:104510008522CF93C82F8091E802813071F040F05E
:10452000823009F045C08C2F0E94D51F81E046C023
:104530000E9474118232F1F504C00E94741182321B
:1045400061F48C2F0E948722811104C08C2F0E945D
:1045500012212CC081E090E029C08C2F0E9485227E
:10456000811123C0C431C9F058F4CB3069F0C03197
:10457000B9F482E08093E80288E30E94D51F15C059
:10458000C93259F0C83361F487E396E00E941806F7
:104590008FEF94E00E94180608C01092E8020CC049
:1045A0008DEF94E00E94180607C081E0817006C07C
:1045B0001092E80280E002C080E0F8CFCF91089529
:1045C000CF93DF9386319C4541F5EB010E94741136
:1045D000982F8A812091020130910301882379F07C
:1045E0009A7A81E009F480E08093E902911102C097
:1045F00069E201C065E3C9010E947A260AC0809180
:10460000E902811102C069E201C065E3C9010E94AB
:104610007C260E94B61180E001C081E0DF91CF913D
:1046200008950F931F93CF93DF93C42FD22FFC01D4
:1046300082818823C9F04093EC020E942027909346
:10464000EB028093EA0280E28C0F883008F057C0BA
:10465000C77081E001C0880FCA95EAF7DF91CF915A
:104660001F910F910C947C098091EC02481330C08B
:104670008091EA029091EB020E943827883C9105D4
:1046800038F510E21D0FCD17B9F080E28C0F88309D
:1046900040F4C77081E001C0880FCA95EAF70E9414
:1046A0008309183028F581E09D2F977001C0880F8D
:1046B0009A95EAF70E947C09802F0E9473091830AE
:1046C000F0F4D77081E001C0880FDA95EAF70AC0EC
:1046D00080E28C0F883098F4C77081E001C0880FA9
:1046E000CA95EAF7DF91CF911F910F910C9483093E
:1046F000802FDF91CF911F910F910C947309DF915F
:10470000CF911F910F9108950F939C01CB01243FEE
:104710004CE5340731F188F4293DFCE53F07D9F039
:104720002A3D4CE5340779F1283D3C45A9F506E2E0
:1047300021EE41EE68ED7CE52BC0263FFCE53F070E
:10474000E1F0A8F0273F3C4539F507E225EE46EEBB
:1047500067EF7CE51DC007E225EE45EE69ED7CE5DF
:1047600017C006E221EE40EE64EF7CE511C007E2DF
:1047700025EE44EE65EF7CE50BC006E221EE42EE4D
:1047800066EF7CE505C008E221E045EE6AED7CE5D8
:104790000E94112380E008C0FC018281882319F067
:1047A0001092EC0201C081E00F9108958EE1489BC8
:1047B00002C08150E1F7489BFECF0895589880E2EF
:1047C0008A95F1F7589A0895FC012AE02A95F1F7A5
:1047D00028E090E080E031E040E14A95F1F7880F71
:1047E000489B02C08160932700C0000040E14A95C9
:1047F000F1F7215089F720E12A95F1F729B100C09E
:10480000000030E13A95F1F7217092272081920F54
:1048100090830895EF92FF920F931F93CF93DF93AE
:104820001F92CDB7DEB719828C017C01E60EF11C18
:104830000E151F0551F00E94D623CE0101960E944D
:10484000E423F80181938F01F3CF81E099819111E5
:1048500080E00F90DF91CF911F910F91FF90EF902B
:104860000895509A589A08955098589AE89AE9E607
:10487000F0E080818C7F80830895615091E001C0D9
:10488000990F6A95EAF720E031E0992361F0492F0A
:10489000482319F0589A232701C0589840E24A95B6
:1048A000F1F79695F2CF222311F0589A01C058984B
:1048B00080E28A95F1F758980895FF920F931F931D
:1048C000CF93DF93EC018C01060F111DC017D107A8
:1048D00041F0F9900E94DE2368E08F2D0E943D2474
:1048E000F5CFDF91CF911F910F91FF9008951F9207
:1048F0000F920FB60F9211240F931F932F933F9394
:104900004F935F936F937F938F939F93AF93BF93D7
:10491000EF93FF93CF93DF931F92CDB7DEB719824A
:104920000E94D623CE0101960E94E423082F06950B
:1049300006950695902F96959570202F2570920FCD
:10494000292F237096959695920F877089135FC0D3
:10495000898181115CC0043008F059C080E18A95DA
:10496000F1F7589A509A82E08A95F1F700C058986A
:1049700088E0089F80011124D801A15FBE4F1696E0
:10498000ED91FC9117973097A9F06091A801709173
:10499000A90114962D913C911597260F371F11965A
:1049A0008D919C911297680F791F13964C911397D4
:1049B0008C910995F801E15FFE4F6381662351F008
:1049C0008091A8019091A90124813581820F931FC4
:1049D0000E945D240E94DE2380E18A95F1F75898B9
:1049E0005098589A80E18A95F1F7F801E15FFE4FFF
:1049F0006081662351F08091A8019091A9012181E5
:104A00003281820F931F0E940A240E94D6230F90A6
:104A1000DF91CF91FF91EF91BF91AF919F918F91D6
:104A20007F916F915F914F913F912F911F910F91C6
:104A30000F900FBE0F901F9018950F931F93CF9359
:104A4000DF93843091050CF06DC0EC01F894509A1E
:104A5000589885E08A95F1F700009C2F96959570FF
:104A60002C2F2570920F892F83709695969523E0B1
:104A7000CC0FDD1F2A95E1F7980F8E01092B0E94BC
:104A8000DE2384E08A95F1F700C068E0802F0E9461
:104A90003D2480E18A95F1F75098589A489902C0D0
:104AA00000C0FCCF87E090E0489B08C0019721F44C
:104AB000509A589A789436C000C0F6CFFE01E15F54
:104AC000FE4F6381662381F08091A8019091A90136
:104AD00024813581820F931F0E940A24811104C012
:104AE000509A589A78941FC00E94D62380E28A95E3
:104AF000F1F75898509A80E18A95F1F7C15FDE4F3F
:104B00006881662351F08091A8019091A9012981C3
:104B10003A81820F931F0E945D240E94DE237894C5
:104B200081E001C080E0DF91CF911F910F91089546
:104B300090932F0280932E0208959093F302809316
:104B4000F20208950E94BE18811103C08091ED0207
:104B50000895E091F202F091F302309721F0019074
:104B6000F081E02D099480E00895EF92FF920F9379
:104B70001F93CF93DF93E091F202F091F30230970D
:104B8000B1F18C010280F381E02D09958091B4028E
:104B900082FF2DC080FF04C083EF99E00E941806B9
:104BA000E80118E08DEEE82E89E0F82E8091B4023D
:104BB00080FF0BC088811F928F93FF92EF920E941B
:104BC000B1060F900F900F900F9011502196111178
:104BD000EDCF8091B40280FF0AC08BEE99E0DF91A7
:104BE000CF911F910F91FF90EF900C941806DF91D9
:104BF000CF911F910F91FF90EF900895E091F202F5
:104C0000F091F302309739F022E0DC012C9304801C
:104C1000F581E02D099408952091F0023091F10280
:104C20002817390771F09093F1028093F002E09118
:104C3000F202F091F302309721F00680F781E02D27
:104C4000099408952091EE023091EF022817390758
:104C500071F09093EF028093EE02E091F202F091F6
:104C6000F302309721F00084F185E02D0994089536
:104C7000FC01329697E080E0915029F021912223A7
:104C8000D9F38F5FF9CF0895662349F0FC0132967E
:104C900008962191621729F0E817F907D1F780E00B
:104CA000089581E008959C01FC0132969FEF80E019
:104CB0004191461789F09F3F19F4411101C0982F87
:104CC0008F5F8630A9F79F3F39F0F901E90FF11D99
:104CD00097FDFA956283089508959C012A5F3F4FDE
:104CE000FC014281461301C012820196821793078C
:104CF000B9F708950C9453260C946D26029626E07D
:104D0000FC0111922A95E9F7089508950C948526DF
:104D100083E08093F4020C948626811102C081E026
:104D200001C082E08093F4020C9486260C948D26B8
:104D300081E08093F4020C9486260C9498260895C2
:104D40000C949F260C94A0260C949F260C949F26CE
:104D50000C949F26CF930E94A6260E942C180E9496
:104D6000A426C0E08C2F0E947716811104C0CF5F6B
:104D7000C830C1F701C081E0CF91089508951F9216
:104D80000F920FB60F9211248F939F93AF93BF93FF
:104D90008091F502811113C080911E0390911F0331
:104DA000A0912003B09121034196A11DB11D8093D4
:104DB0001E0390931F03A0932003B0932103BF9180
:104DC000AF919F918F910F900FBE0F901F901895EC
:104DD00080912603843031F10E9491071092F502F0
:104DE00020E488E190E00FB6F894A89580936000E5
:104DF0000FBE2093600083B7817F846083BF83B739
:104E0000816083BF7894889583B78E7F83BF0FB608
:104E1000F894A8958091600088618093600010925A
:104E200060000FBE08950E941F0C0C94950782E04D
:104E300084BD93E095BD9AEF97BD80936E00089571
:104E40002FB7F89480911E0390911F03A091200327
:104E5000B09121032FBF08952FB7F89460911E03DE
:104E600070911F0380912003909121032FBF08951B
:104E70009C014FB7F89480911E0390911F03A0915D
:104E80002003B09121034FBF821B930B0895CF9253
:104E9000DF92EF92FF922FB7F894C0901E03D0904C
:104EA0001F03E0902003F09021032FBFA70196017C
:104EB000261B370B480B590BCA01B901FF90EF9025
:104EC000DF90CF90089578941F920F920FB60F92B3
:104ED00011248F939F93AF93BF9380911E03909162
:104EE0001F03A0912003B09121030196A11DB11DC4
:104EF00080931E0390931F03A0932003B09321037C
:104F0000BF91AF919F918F910F900FBE0F901F9007
:104F1000189581E08093E00080E28093D8001092A1
:104F2000C9008FE19EE40197F1F700C0000087E01F
:104F300090EBDC0180932F0390933003A093310317
:104F4000B09332039CE088E10FB6F894A895809363
:104F500060000FBE90936000FFCF8091040308951E
:104F6000089522E02093E9002FEF3091E8002150CE
:104F700035FD06C035ED3A95F1F700002111F5CF6A
:104F80002091E80025FF0BC040E050E066E070E0B3
:104F90000E94992A8091E8008E778093E800089516
:104FA000CF93DF9321E02093E9002FEF3091E800C9
:104FB000215035FD06C035ED3A95F1F7000021117D
:104FC000F5CF2091E80025FF14C0EC0140E050E04F
:104FD00068E070E00E94992A8091E8008E778093C3
:104FE000E80088E0FE01ACEFB2E001900D928A95F6
:104FF000E1F7DF91CF9108958093F8027093FA0260
:105000006093F90280912603843001F582E0809359
:10501000E9008FEF9091E800815095FD06C095ED75
:105020009A95F1F700008111F5CF8091E80085FF96
:105030000DC040E050E063E070E088EF92E00E9435
:10504000992A8091E8008E778093E8000895BC014A
:1050500084E00C94FC27BC0183E00C94FC2789E1DC
:105060009AE00E94180680912503811109C00E94D0
:105070002A2C0E94872C8091E20084608093E200B9
:10508000089585E19AE00E9418061092250308957C
:1050900081E19AE00E9418060C949D268DE09AE02A
:1050A0000E9418066091220381E0611101C080E036
:1050B0000C94882689E09AE00E94180690912603B5
:1050C00081E0943009F080E0609122030C948D26F9
:1050D0002091F7022F5F822F62E30E94412F9923D4
:1050E00019F02093F70208951092F7028091FB02C5
:1050F000882371F180912603843041F58091E90085
:105100008F702091EC00922F917020FD90E8892BF8
:1051100093E09093E9009091EB0090FF14C0909180
:10512000EE0097FF10C09091E80095FF03C0109229
:10513000F100F9CF9091E80090FF05C09091E80050
:105140009E779093E8008F708093E9001092FB02A5
:10515000089542E061EC81E00E94A32B42E261EC01
:1051600082E00E94A32B42E261EC83E00E94A32B29
:105170009091260381E0943009F080E06091220351
:105180000C94962680912803833009F461C030F492
:10519000813071F0823009F49AC008958A3009F4A0
:1051A00086C08B3009F46CC0893009F0A8C020C0DB
:1051B00080912703813A09F0A2C08091E800877F9F
:1051C0008093E80080912B0390912C03892B21F48C
:1051D00068E08CEF92E003C060E080E090E070E077
:1051E0000E94E42A8091E8008B778093E80008957C
:1051F00080912703813209F082C080912B03909126
:105200002C03029708F07BC08091E800877F809391
:10521000E8008091E80082FD05C08091260381119D
:10522000F8CF6DC02091F3008091F20090E0922BB6
:10523000029731F48091F100813011F0863021F431
:105240008091F100809304038091E8008B7753C034
:1052500080912703813A09F052C080912B039091ED
:105260002C03892B09F04BC08091E800877F809345
:10527000E8008091E80080FFFCCF80913B0136C0C0
:10528000809127038132D9F580912B0390912C03D3
:10529000892BA9F58091E800877F8093E8000E9420
:1052A000D82B8091290380933B010C941F0C809193
:1052B0002703813221F58091E800877F8093E80001
:1052C0000E94D82B80912A03809305030895809132
:1052D0002703813AA1F48091E800877F8093E8005A
:1052E0008091E80080FFFCCF809105038093F1005E
:1052F0008091E8008E778093E8000C94D82B089575
:105300009FB7F8941092FB029FBF909126039430B0
:1053100009F057C09091E9009F703091EC00232F65
:10532000217030FD20E8922B23E02093E9002091AA
:10533000EB0020FF43C02091EE0027FF3FC02091EB
:10534000F602222321F02091E80025FF37C01092B9
:10535000F60226E03091E80035FD15C030912603B5
:10536000343061F53091EB0035FD28C0215021F437
:1053700081E08093F60222C0EFE9FFE03197F1F778
:1053800000C00000E7CF8093F1008091E80085FD28
:105390000AC08091E80080FFFCCF8091E8008E7702
:1053A0008093E80006C08FB7F89421E02093FB02B9
:1053B0008FBF9F709093E90080E008959F70909355
:1053C000E9008FEF089584B7877F84BF0FB6F89404
:1053D000A8958091600088618093600010926000C1
:1053E0000FBE90E080E80FB6F89480936100909330
:1053F00061000FBE0C9498260E942A2C0E94872CD4
:10540000E2EEF0E080818460808378940C941B2F1E
:105410008FE291E00C949D25809126038530C9F49C
:1054200085E09AE00E94180680912603853079F481
:105430000E94E826809124038823B1F30E94AA26C3
:10544000882391F30E94832A0E941F0CEDCF0C94B5
:105450001327089508950C942D2A292F33272330DC
:105460003105C9F060F42130310581F02230310579
:1054700009F041C08BE590E029E53AE040C02132D7
:105480003105E1F02232310531F135C082E190E0A1
:1054900024EB3AE034C099278130910549F028F097
:1054A000029749F5EDE1FAE005C0E5E5FAE002C052
:1054B000EDE2FAE0849190E09F0121C06330710534
:1054C000D0F4660F771FFB01E85DFD4F208131812D
:1054D00089E090E014C06330710568F4FB01EE0FC1
:1054E000FF1FEE5DFD4F20813181FB01E15EFD4F2D
:1054F000808190E004C080E090E020E030E0FA019C
:1055000031832083089580E189BD82E189BD09B49A
:1055100000FEFDCF8091D8008F7D8093D8008091D0
:10552000E00082608093E0008091E00081FDFCCF8C
:105530000895CF92DF92EF92FF920F931F93CF9334
:10554000DF93EC018B017A010E94F72B811133C0AC
:10555000E114F10439F0F70180819181081B190BE6
:10556000C80FD91FC12CD12C0115110519F180913B
:10557000E80085FD16C08091E8008E778093E800F2
:10558000E114F10449F0F70180819181C80ED91E20
:10559000D182C08285E00FC00E94F72B882321F3BF
:1055A0000AC089918093F10001501109FFEFCF1AD1
:1055B000DF0ADACF80E0DF91CF911F910F91FF904A
:1055C000EF90DF90CF90089520912D0330912E031E
:1055D0002617370748F06115710539F42091E80066
:1055E0002E772093E80001C0B901FC0120E061158D
:1055F000710579F1809126038823F1F18530F1F16D
:105600008091E80083FD3CC08091E80082FD2EC0BF
:105610008091E80080FFEBCF2091F3008091F200B1
:1056200090E0922B6115710551F08830910538F4A6
:1056300021912093F100615071090196F3CF21E08F
:10564000089709F020E08091E8008E778093E800C9
:10565000CECF2111CFCF0AC080912603882361F0DD
:10566000853061F08091E80083FD0AC08091E800F8
:1056700082FFF2CF80E0089582E0089583E00895EC
:1056800081E0089520912D0330912E0326173707CE
:1056900048F06115710539F42091E8002E772093C8
:1056A000E80001C0B901FC0120E06115710591F12C
:1056B00080912603882309F440C0853009F43FC057
:1056C0008091E80083FD3DC08091E80082FD2FC0FD
:1056D0008091E80080FFE9CF2091F3008091F200F3
:1056E00090E0922B6115710559F08830910540F4D6
:1056F00024912093F1003196615071090196F2CF07
:1057000021E0089709F020E08091E8008E778093EF
:10571000E800CBCF2111CCCF0AC08091260388238B
:1057200061F0853061F08091E80083FD0AC08091CE
:10573000E80082FFF2CF80E0089582E0089583E0E0
:10574000089581E00895982F973068F59093E900C7
:10575000981739F07091EC002091ED005091F00015
:1057600003C0242F762F50E021FD02C09F5FECCFB5
:105770003091EB003E7F3093EB003091ED003D7FA8
:105780003093ED003091EB0031603093EB0070937B
:10579000EC002093ED005093F0002091EE0027FDE7
:1057A000E5CF80E008958F708093E90081E008954F
:1057B0008091270387FF11C08091E80082FD05C01A
:1057C000809126038111F8CF11C08091E8008B777A
:1057D0000BC080912603882349F08091E80080FF68
:1057E000F8CF8091E8008E778093E80008952091AB
:1057F000E4003091E50095E64091EC00842F817043
:1058000040FF23C08091E80080FD1DC080912603E9
:10581000882399F0853099F08091EB0085FD11C0C7
:105820004091E4005091E5002417350729F3915089
:1058300011F09A01E1CF84E0089582E0089583E0B9
:10584000089581E0089580E008954091E80042FFC6
:10585000DDCF08950E94982C0E94A02CE0EEF0E08D
:10586000808181608083E8EDF0E080818F778083A4
:1058700019BCA7EDB0E08C918E7F8C9380818F7ED8
:1058800080831092250308950F931F93CF93DF9386
:105890000E94982C0E94A02CC8EDD0E088818F77C0
:1058A000888388818068888388818F7D888319BCFC
:1058B00010922603109222031092240310922303C5
:1058C00000EE10E0F80180818B7F80838881816009
:1058D000888342E060E080E00E94A32BE1EEF0E0EC
:1058E00080818E7F8083E2EEF0E080818160808322
:1058F000808188608083F80180818E7F80838881A9
:1059000080618883DF91CF911F910F910895E8ED19
:10591000F0E080818F7E8083E7EDF0E08081816020
:10592000808384E082BF81E0809325030C94442C23
:10593000E8EDF0E080818E7F80831092E200089590
:105940001092DA001092E10008951F920F920FB6A4
:105950000F9211242F933F934F935F936F937F93F5
:105960008F939F93AF93BF93EF93FF938091E10049
:1059700082FF0BC08091E20082FF07C08091E100AE
:105980008B7F8093E1000E9468288091DA0080FF7D
:105990001FC08091D80080FF1BC08091DA008E7FED
:1059A0008093DA008091D90080FF0DC080E189BD2D
:1059B00082E189BD09B400FEFDCF81E0809326031A
:1059C0000E942F2805C019BC109226030E9441286E
:1059D0008091E10080FF19C08091E20080FF15C036
:1059E0008091E2008E7F8093E2008091E2008061EE
:1059F0008093E2008091D80080628093D80019BC27
:105A000085E0809326030E944E288091E10084FF68
:105A100030C08091E20084FF2CC080E189BD82E12A
:105A200089BD09B400FEFDCF8091D8008F7D8093A1
:105A3000D8008091E1008F7E8093E1008091E200A8
:105A40008F7E8093E2008091E20081608093E2008B
:105A500080912203882311F084E007C08091E30045
:105A600087FD02C081E001C083E0809326030E948D
:105A70005A288091E10083FF29C08091E20083FFD2
:105A800025C08091E100877F8093E10082E08093D0
:105A90002603109222038091E1008E7F8093E10023
:105AA0008091E2008E7F8093E2008091E20080612D
:105AB0008093E20042E060E080E00E94A32B8091AE
:105AC000F00088608093F0000E944828FF91EF91D9
:105AD000BF91AF919F918F917F916F915F914F9106
:105AE0003F912F910F900FBE0F901F9018951F920E
:105AF0000F920FB60F9211242F933F934F935F9302
:105B00006F937F938F939F93AF93BF93CF93DF93C5
:105B1000EF93FF93C091E900CF708091EC00D82FF4
:105B2000D17080FDD0E81092E9008091F000877F6D
:105B30008093F00078940E94BB2D1092E900809130
:105B4000F00088608093F000CD2BCF70C093E90007
:105B5000FF91EF91DF91CF91BF91AF919F918F9185
:105B60007F916F915F914F913F912F910F900FBE59
:105B70000F901F9018951F93CF93DF93CDB7DEB78B
:105B8000AA970FB6F894DEBF0FBECDBFE7E2F3E0F1
:105B90008091F100819323E0EF32F207C9F70E9470
:105BA000C2288091E80083FF2EC180912703909145
:105BB0002803492F50E04A30510508F024C1FA016A
:105BC000EE59FF4F0C94612F803821F0823809F094
:105BD0001AC108C08091230390912403992389F06E
:105BE00082600FC080912B038F70873008F00BC14B
:105BF0008093E9008091EB0085FB882780F9109263
:105C0000E9009091E800977F9093E8008093F1007D
:105C10001092F100D1C0282F2D7F09F0F4C0882305
:105C200019F0823061F0EFC080912903813009F0D2
:105C3000EAC0933009F080E0809324032EC0809165
:105C4000290381112AC080912B038F702FEF280F19
:105C5000263008F0D8C08093E9002091EB0020FFA7
:105C60001CC0933021F48091EB00806214C09091AD
:105C7000EB0090619093EB0021E030E0A90102C0BD
:105C8000440F551F8A95E2F74093EA001092EA000C
:105C90008091EB0088608093EB001092E900809186
:105CA000E800877F8093E8000E94D82BACC0811168
:105CB000AAC0109129031F778091E3008078812B7F
:105CC0008093E3008091E800877F8093E8000E9442
:105CD000D82B8091E80080FFFCCF8091E3008068A2
:105CE0008093E300111102C082E001C083E0809341
:105CF000260389C08058823008F085C0809129032E
:105D000090912A038C3D53E0950779F583E08A83CF
:105D10008AE289834FB7F894DE01139620E03EE0D3
:105D200051E2E32FF0E050935700E49120FF03C0CD
:105D3000E295EF703F5FEF708E2F90E0EA3010F049
:105D4000C79601C0C0968D939D932F5F243149F76C
:105D50004FBF8091E800877F8093E8006AE270E09F
:105D6000CE0101960E94E42A16C060912B03709127
:105D70002C03AE014F5F5F4F0E942B2ABC01892B81
:105D800009F441C09091E800977F9093E8008981E1
:105D90009A810E94422B8091E8008B778093E800E3
:105DA00032C0803881F58091E800877F8093E800D9
:105DB000809122038093F1008091E8008E7772CF6A
:105DC000811121C08091290390912A03992702977C
:105DD000D4F48091E800877F8093E80080912903C4
:105DE000809322030E94D82B80912203811106C048
:105DF0008091E30087FD02C081E001C084E08093D0
:105E000026030E94A9288091E80083FF0AC08091A0
:105E1000E800877F8093E8008091EB0080628093A8
:105E2000EB00AA960FB6F894DEBF0FBECDBFDF9190
:105E3000CF911F910895CF93809126038823A1F0DD
:105E4000C091E900CF709091EC00892F817090FD96
:105E500080E8C82B1092E9008091E80083FD0E9441
:105E6000BB2DCF70C093E900CF9108950E942A2CDA
:105E70001092260308958091E300881F8827881FC9
:105E80000895991B79E004C0991F961708F0961B96
:105E9000881F7A95C9F78095089597FB072E16F409
:105EA000009407D077FD09D00E94672F07FC05D02A
:105EB0003EF4909581959F4F0895709561957F4F21
:105EC0000895EE0FFF1F0590F491E02D0994AA1B91
:105ED000BB1B51E107C0AA1FBB1FA617B70710F0D5
:105EE000A61BB70B881F991F5A95A9F78095909507
:105EF000BC01CD010895FB01DC0104C08D9101902E
:105F0000801921F441505040C8F7881B990B08951F
:105F1000FB01DC0102C001900D9241505040D8F7C6
:105F20000895F999FECF92BD81BDF89A992780B561
:105F30000895A8E1B0E042E050E00C94C52F262F70
:105F4000F999FECF92BD81BDF89A019700B402166F
:105F500039F01FBA20BD0FB6F894FA9AF99A0FBE1D
:105F600008950396272F0E94A02F0E949F2F252F70
:105F70000E94A02F242F0C94A02F0196272F0E945F
:105F8000A02F0C949F2FDC01CB01FC01F999FECFCF
:105F900006C0F2BDE1BDF89A319600B40D924150B1
:0A5FA0005040B8F70895F894FFCFC1
:105FAA00C8009A02C6F631306766979694F00100E7
:105FBA0000000100000000000000040100000004CD
:105FCA0005000000000000280850011E0A1401AD57
:105FDA0027D027B1272B282728B0270135973494B3
:105FEA00963631303332E200E900EA00B500B600F5
:105FFA00B700CD008301CC008A01920194012102ED
:10600A00230224022502260227022A02B300B40030
:10601A006F007000818283E200E900EA00B500B6F1
:10602A0000B700CD008301CC008A019201940121BE
:10603A0002230224022502260227022A02B300B4FE
:10604A00006F007000818283BD02736C6176655FA8
:10605A006D61747269780073796E635F74696D65D6
:10606A0072003F3F3F006D6B5F64656C6179006D44
:10607A006B5F696E74657276616C006D6B5F6D61E2
:10608A00785F7370656564006D6B5F74696D655FD9
:10609A00746F5F6D6178006D6B5F776865656C5FC3
:1060AA006D61785F7370656564006D6B5F776865B5
:1060BA00656C5F74696D655F746F5F6D61780040D0
:0E60CA007B22630BE80AC60A6B0A840A9D0A51
:00000001FF
